:10000000FF23831690001F3085000B30870083127A
:10001000E3200024B50000308A00350EBD00BD0C81
:100020003D0C0339143E82001828E128E128772886
:1000300000308A00350CBD00BD0C3D0C0739213E57
:10004000820029285328762876287628762876284C
:1000500076285F1500308A0035082F3E8200372849
:100060003B283E284D284128442847284A2828086C
:100070002906B6004E282908B6004E282808B600E2
:100080004E282B08B6004E282C08B6004E282D0806
:10009000B6004E282E08B6004E285F115F1D52286C
:1000A00036082924762800308A00350CBD00BD0CA6
:1000B0003D0C07395C3E8200642866287528752847
:1000C00069286C286F287228E32075280024A9006D
:1000D00075280024AB0075280024AC007528002486
:1000E000AD0075280024AE0075287628E128003080
:1000F0008A00350CBD00BD0C3D0C0739803E8200E6
:10010000E128E128E128E128E12888289528B2287B
:1001100011303507031D94280030B600AA18361494
:100120002A18B61436082924E12800308A0007303E
:1001300035059B3E8200A328A328A328A328AA282C
:10014000AA28AE28AE282A10B5182A14AA103518E5
:10015000AA14B128AA103518AA14B1282A103518E3
:100160002A14E12800308A0007303505B83E8200A5
:10017000C028C428C828CD28D028D528D828DD28CC
:100180008316FC309007E028831604309007E0289F
:100190008316100883122924E02800302924E0283F
:1001A0003108DA212924B10AE0280030B100E02822
:1001B000300829240030B000E028300A031DB00ABE
:1001C000E12883120928073099000030B1000B3074
:1001D000BE003108243E840000308000B10ABE0B0E
:1001E000E9280030B3000030B4000030B200003025
:1001F000B0000030B100003464000030A800051CDD
:100200002814851CA814051D2815851DA815051E74
:100210002816851EA816071C2817871CA81739083A
:10022000B80028082906B9000F303906BA00390885
:100230003806BB002B083A05BF002C083905BF045F
:100240003B0839052D05BF043B083A052E053F0440
:10025000031DAA14AA182F292D292E2935292A1859
:100260003329000035292A10071101308A0033088C
:100270003A3E82006129CD29CD2967296F29CD29F0
:1002800067296F29CD2967296F29CD2967296F290A
:10029000CD2967296F29CD2967296F29CD2967299C
:1002A0006F29CD2967296F29CD2967297629CD297D
:1002B0007D2985298F299729A229AC29B629BC290E
:1002C000C62907120230FF3E031D6329D3293218C5
:1002D0000716321C07126C296D290000D329B20CB5
:1002E000B213B217732974297529D329340CB200BB
:1002F000B2137A297B297C29D3293208243E840031
:100300000008B20083298429D329341C892988292B
:100310008C29B20E0F30B2058D290000D3290F3081
:100320003205303EB200942995290000D329393096
:1003300032020319031003189F290000A129073076
:10034000B207D329163034020318A8290000AA29BD
:100350000D30B200AB29D329173034020318B2296B
:100360000000B4298830B200B529D329B40A02307C
:10037000FF3E031DB829D329183034020318C229BF
:100380000000C4290030B400C529D329FF30B300D0
:10039000C929CA29CB290000D3290230FF3E031DF9
:1003A000CE290000D3298312B30A0E30FF3E031D6D
:1003B000D6290034BC002E303C0203190310031868
:1003C0002F2A02308A003C08003E82000000000014
:1003D000000000000000000000000000000000001D
:1003E000000000000000000000000000000000000D
:1003F00000000000000000000000000000000000FD
:100400000134003420340134033401340034003426
:10041000003400340034003400340034003400343C
:10042000003400340034003400340034003400342C
:10043000083453347734693474346334683438346A
:1004400045340D344D346F346E3464346F342D3490
:10045000743472346F346E346934633473340034FA
:0207FE00A03425
:10080000DF145F14871D062CFC20022CDF10071557
:10081000FC20FC20FC200030A1000E2C0F2C102C02
:1008200000000830C000FC20A10CA1138719A117FB
:10083000FC20FC201B2C1C2CC00B132CFC20FC20AF
:10084000212C00002508A4002108A5000715210877
:100850000800A3002608A7002308A6005F1C362C6A
:100860005F100A30C100FC20C10B332C0711FC20A3
:10087000FC20FC200230FF3E031D3B2C0830C10051
:1008800023180715231C0711A30CA313FC20FC201D
:10089000FC204A2CC10B402C0715FC20FC20FC201E
:0C08A0000230FF3E031D512C552C00348B
:02400E009431EB
:00000001FF
